:020000040800F2
:10000000400C0020F5020008BB100008E90E0008B3
:10001000B9100008EB040008851200080000000079
:100020000000000000000000000000003502000891
:10003000ED0400080000000091020008BD10000857
:100040000F0300080F0300080F0300080F03000848
:100050000F0300080F0300080F0300080F03000838
:100060000F0300080F0300080F0300080F03000828
:100070000F0300080F0300080F0300080F03000818
:100080000F0300080F0300080F0300080000000022
:100090000000000000000000000000000F03000846
:1000A0000F0300080F0300080F0300080F030008E8
:1000B0000F0300080F0300080F0300080F030008D8
:1000C0000F0300080F0300080F0300080F030008C8
:1000D0000F0300080F0300080F03000800000000D2
:1000E0000F0300080F0300080F03000800000000C2
:1000F0000000000000000000000000000F030008E6
:10010000000000000F0300080F0300080F030008A1
:1001100000000000000000000000000000000000DF
:100120000F0300080F0300080F0300080F03000867
:100130000F030008000000000000000000000000A5
:100140000000000000000000000000000F03000895
:100150000F0300080F0300080F0300080F03000837
:100160000F0300080F03000800000000000000005B
:10017000000000000000000000000000000000007F
:10018000000000000F030008000000000000000055
:100190000F03000800F002F800F03CF80AA090E815
:1001A000000C82448344AAF10107DA4501D100F032
:1001B00031F8AFF2090EBAE80F0013F0010F18BFC3
:1001C000FB1A43F0010318472813000048130000EE
:1001D000103A24BF78C878C1FAD8520724BF30C873
:1001E00030C144BF04680C60704700000023002445
:1001F00000250026103A28BF78C1FBD8520728BF37
:1002000030C148BF0B6070471FB501F05FF91FBDDB
:1002100010B510BD00F02FF91146FFF7F5FF01F002
:1002200043F800F04DF903B4FFF7F2FF03BC00F010
:1002300055F900002C4B19680868B0E8F04F80F3BE
:100240000988BFF36F8F4FF0000080F3118870476B
:100250000000000008480068006880F308884FF03C
:10026000000080F3148862B661B6BFF34F8FBFF30E
:100270006F8F00DF00BF00BF08ED00E0DFF80C006B
:10028000016841F470010160704700BF88ED00E033
:10029000EFF30980BFF36F8F134B1A681EF0100F36
:1002A00008BF20ED108A20E9F04F106009B44FF02C
:1002B000500080F31188BFF34F8FBFF36F8F01F0B1
:1002C0004BF84FF0000080F3118809BC19680868EA
:1002D000B0E8F04F1EF0100F08BFB0EC108A80F3AA
:1002E0000988BFF36F8F704710000020EFF305807F
:1002F000704700000948804709480047FEE7FEE7CD
:10030000FEE7FEE7FEE7FEE7FEE7FEE7FEE7FEE7C5
:1003100004480549054A064B70470000691100086A
:100320009501000840060020400C002040080020F5
:100330004008002053EA020C00F069802DE9F04BE0
:100340004FF00006002B1FBFB3FA83F503FA05F444
:1003500024FA05F65E4012BF1643B2FA82F502FA9D
:1003600005F4C5F120051EBF22FA05FC44EA0C0481
:10037000203556EA044C4FEA144418BF641C4FF071
:1003800000084FF00009904271EB030C39D30029AB
:1003900019BFB1FA81F701FA07F6B0FA80F700FA4F
:1003A00007F6C7F120071EBF20FA07FC46EA0C0635
:1003B0002037B6FBF4FCA7EB0507103F07F01F0B37
:1003C000CBF120060CFA0BFB2CFA06F644BFB34621
:1003D0000026202FA4BF5E464FF0000B5BEA060C00
:1003E00008BF4FF0010B19EB0B09ABFB027C48EB8C
:1003F0000608C01B06FB02CC0BFB03CC71EB0C0107
:10040000C1E70B46024641464846BDE8F08B13B5AE
:100410004FF000004FF00001AFF30080BDE81C403A
:1004200070474FF0000200B51346944696462039B7
:1004300022BFA0E80C50A0E80C50B1F12001BFF49D
:10044000F7AF090728BFA0E80C5048BF0CC05DF803
:1004500004EB890028BF40F8042B08BF704748BF51
:1004600020F8022B11F0804F18BF00F8012B7047C5
:10047000704770477047754600F02CF8AE4605008F
:100480006946534620F00700854618B020B5FFF7AF
:100490003FFFBDE820404FF000064FF000074FF04F
:1004A00000084FF0000B21F00701AC46ACE8C00992
:1004B000ACE8C009ACE8C009ACE8C0098D4670479B
:1004C00010B50446AFF300802046BDE81040FFF7AA
:1004D000AABE000000487047DC0500200149182032
:1004E000ABBEFEE7260002007047FEE7704772B61B
:1004F000FEE7000070B5044600F004F90546601CF4
:1005000002D004480078044400F0FCF8401BA042EC
:10051000FAD370BD000000202DE9F84FDFF8B8A134
:10052000002201240AF1040B03254FF00F090BF1FF
:10053000040E00BF0B6804FA02F63340B34273D1D5
:100540000F7907F00307012F01D0022F16D187681A
:100550004FEA420805FA08FC27EA0C07D1F80CC05C
:100560000CFA08FC4CEA070CC0F808C04768B7430F
:100570000E79C6F3001696403E4346600E79F64368
:10058000B6070DD0C768560005FA06FC27EA0C0727
:10059000D1F808C00CFA06FC4CEA070CC0F80CC0F5
:1005A0000E7906F00306022E10D1D60800EB86085D
:1005B000D8F8206057074FEAD76C09FA0CF7BE430A
:1005C0000F6907FA0CF73743C8F8207006684FEA3E
:1005D000420C05FA0CF7BE430F7907F0030707FA40
:1005E0000CF7374307604E6816F4403F6DD03B4E22
:1005F000376847F480473760366822F0030706F40F
:1006000080460096364E07EB060CDCF80868970724
:100610003F0F09FA07F826EA0806DFF8C8804045C8
:1006200003D14FF000081EE04FE0DFF8BC804045EA
:1006300002D14FF0010816E0DFF8B080404502D14A
:100640004FF002080FE0DFF8A880404502D14FF0DC
:10065000030808E0DFF89C80404502D14FF0040811
:1006600001E04FF0070808FA07F848EA0608CCF856
:100670000888DAF800605746D1F804C09E435FEA64
:10068000CC3C00D51E433E60DBF800605F46D1F8ED
:1006900004C09E435FEA8C3C00D51E433E60DEF8FA
:1006A00000607746D1F804C09E435FEACC2C00D5A9
:1006B0001E433E60084F0C373E68D1F804C09E438D
:1006C0005FEA8C2C00D51E433E60521C102AFFF4BA
:1006D00031AFBDE8F88F0000003C014044380240D3
:1006E00000300140000002400004024000080240C7
:1006F000000C0240001002400AB1816170470904F9
:10070000FBE70000014880687047000000000020FF
:10071000024881680278114481607047000000201F
:100720000B4810B5016841F400710160016841F4A3
:1007300080610160016841F480710160032000F074
:1007400065F80F2000F006F800F024F8002010BD36
:10075000003C024070B50D4D04464FF47A71287884
:10076000B1FBF0F00A490968B1FBF0F000F000FBC2
:1007700048B9102C07D200222146501E00F026F85E
:1007800000206C6070BD012070BD000000000020E2
:100790000C0000200C4882B0016841F480410160E7
:1007A000006800F4804000900748001F016841F095
:1007B000805101600068002200F0805000900F21FD
:1007C000901E02B000F002B844380240F0B40E4B64
:1007D0001B680C46C3F30223C3F10705042D00D99F
:1007E0000425191D072901D2002300E0DB1E012684
:1007F00006FA05F1491E214099409E40761E16409A
:100800003143F0BC00F03FBD0CED00E0064900F0C4
:10081000070208684FF6FF03184040EA0220034A27
:1008200010430860704700000CED00E00000FA057E
:100830002DE9F0470E46050065D0DFF81481D8F8A1
:100840000000F7B200F00700B04207D288F800704D
:10085000D8F8000000F00700B04254D128683D4CA1
:10086000810712D5400703D5206840F4E05020608E
:100870002878000703D5206840F460402060206895
:10088000A96820F0F000084320602878C0072DD028
:10089000304968680839012812D0022813D003288B
:1008A00011D00968890700292DDA216821F0030198
:1008B00001432160FFF726FF814641F2883A0EE0AE
:1008C00009688903EFE709688901ECE7FFF71AFF78
:1008D000A0EB0901514502D90320BDE8F08720684B
:1008E000696800F00C00B0EB810FEFD1D8F8001070
:1008F000404601F00701B14207D90770006800F0D7
:100900000700B04201D00120E7E72878400705D56D
:100910002068E96820F4E050084320602878000748
:1009200006D52068296920F4604040EAC1002060B3
:1009300000F038F82168084AC1F30311515CC8403F
:100940000649086006480068FFF704FF0020C4E776
:10095000003C024008380240D61400080C00002079
:10096000040000200448054900680968044AC1F3EE
:100970008221515CC84070470C00002008380240BA
:10098000E61400080448054900680968044AC1F3F0
:100990004231515CC84070470C00002008380240CA
:1009A000E6140008154810B5006810F00C02144851
:1009B00013D04110042A0FD0082A0ED10F4C241F47
:1009C0002268236802F03F025B0207D52068C0F36B
:1009D0008810A0FB010106E0084610BD2168C1F3A4
:1009E0008811A1FB00010023FFF7A4FC2168C1F3DB
:1009F0000141491C4900B0FBF1F010BD083802402C
:100A00000024F4002DE9F84F04006ED02078DFF8C0
:100A10004C93C007A9F104054AD009F1040001680C
:100A2000C1F38101012908D00068C0F381000228C8
:100A30000AD1D9F80000400206D52868800337D5CE
:100A400060680028E1D033E06068B0F5803F10D0E6
:100A5000B0F5A02F286810D020F4803028602868D6
:100A600020F4802028606068A8B1FFF74BFE06469E
:100A70000DE0286840F48030F4E740F480202860DE
:100A8000F7E700BFFFF73EFE801B642873D8286895
:100A90008003F7D50CE0FFF735FE064605E000BF02
:100AA000FFF730FE801B6428F0D828688003F7D455
:100AB0002078DFF8AC8280074FF0000A3ED5A748C7
:100AC000001D016811F00C0F08D00068C0F3810010
:100AD00002280BD1D9F80000400207D4286880070B
:100AE00016D5E068012800D112E033E1E068B8B122
:100AF0000120C8F80000FFF705FE064605E000BF2C
:100B0000FFF700FE801B0228C0D828688007F7D5B1
:100B10002868216920F0F80040EAC10028600DE053
:100B2000C8F800A0FFF7EEFD064604E0FFF7EAFD77
:100B3000801B02281FD828688007F7D42078000778
:100B400022D5864F87486169703771B101210160F4
:100B5000FFF7D8FD064604E0FFF7D4FD801B02280E
:100B600009D838688007F7D50EE0C0F800A0FFF775
:100B7000C9FD064605E082E0FFF7C4FD801B0228A0
:100B80007DD838688007F7D42078400768D5DFF82B
:100B9000CCB100270BF13C0BDBF80000C0000BD4FC
:100BA000DBF8001041F08051CBF80010DBF80000BA
:100BB000012700F0805000906B4E3068C00510D4C3
:100BC000306840F480703060FFF79CFD009005E0D5
:100BD000FFF798FD0099401A022850D83068C005E8
:100BE000F6D55E4EA0686C3601280FD00528306817
:100BF00010D020F001003060306820F00400306038
:100C0000A068B8B1FFF77EFD00900FE0306840F0BB
:100C10000100F4E740F004003060F7E7FFF772FDF1
:100C20000099411A41F28830814266D830688007C5
:100C3000F4D50EE0FFF766FD009007E0FFF762FDD8
:100C40000099411A41F28830814256D830688007B5
:100C5000F4D42FB1DBF8001021F08051CBF8001054
:100C6000A069C8B33D49091D0968C1F38101022982
:100C70004AD00228504607D0C8F8600000E03CE0A7
:100C8000FFF740FD04463BE04746C8F86000FFF729
:100C900039FD064605E000BFFFF734FD801B022842
:100CA0002BD828688001F7D4D4E907010843A16A4A
:100CB0002E4A490802EB0141626A41EA8211084367
:100CC00094F82C1040EA0161C9F800100120386640
:100CD000FFF718FD044606E03EE000BFFFF712FDF7
:100CE000001B022809D828688001F7D534E000BF2E
:100CF000FFF708FD001B022802D90320BDE8F88F8A
:100D000028688001F4D427E00128F7D0D9F8000042
:100D1000E26900F4800191421CD1226A00F03F0197
:100D2000914217D147F6C071626A0140B1EB821F50
:100D300010D1A26A4FF0FF3300F4403103EB5202AE
:100D4000B1EB024F06D194F82C1000F07060B0EBBC
:100D5000016F01D00120D1E70020CFE70438024025
:100D600000004742800E4742007000400000FFFF35
:100D700010B5401EB0F1807F01D3012010BD4FF0AF
:100D8000E02460610F21601700F07DFA0020A0616F
:100D900007202061002010BD70B5040004D094F835
:100DA0003D00002510B106E0012070BD84F83C50E4
:100DB000204600F023F8242084F83D002068C16814
:100DC00021F40051C160204600F0D6F92068016985
:100DD00021F4904101612068416921F02A014161BB
:100DE0002068C16841F40051C1602564202084F866
:100DF0003D0084F83E00002070BD0000F0B587B0D3
:100E0000044614216846FFF70CFB3249DFF8C0C0E6
:100E1000276800222F4B14390224032507262E4869
:100E2000674517D11F6847F010071F601B6803F064
:100E3000100305930B6843F001030B60096802AFD0
:100E400001F0010105916902CDE9001487E8640011
:100E500069461CE0DFF884C067451CD11D4B1B1F91
:100E60001F6847F400371F601B6803F400330593C5
:100E70000B6843F001030B60096802AB01F001014C
:100E800005910C21CDE9001483E864006946FFF761
:100E900043FB07B0F0BD12488742FAD1186840F012
:100EA00020001860186800F020000590086840F0E5
:100EB000040008600868029200F004000590C02059
:100EC000CDE900040820CDE9035069460548DEE776
:100ED000001001404438024000000240004400403D
:100EE0000014014000080240FEE700002DE9F04731
:100EF00086B014216846FFF794FA40480024016840
:100F000041F004010160016801F0040105910168EC
:100F100041F080010160016801F0800105910168E4
:100F200041F001010160016801F0010105910168D2
:100F300041F002010160016801F0020105910168C0
:100F400041F0080101600068012200F008002C4F08
:100F50005503059029463846FFF7CEFBDFF8A480FD
:100F60000022D0214046FFF7C7FBDFF89C904FF2EC
:100F7000FF76002231464846FFF7BEFBDFF88CA023
:100F8000002204215046FFF7B7FB00950125CDE96B
:100F90000154694638460394FFF7BEFA2120CDE993
:100FA0000004694640460294FFF7B6FA022000901A
:100FB000CDE9010469464046CDE90345FFF7ACFAA7
:100FC000D0200090CDE90154694640460394FFF7D4
:100FD000A3FA0096CDE90154694648460394FFF709
:100FE0009BFA04200090CDE90154694650460394D1
:100FF000FFF792FA06B0BDE8F087000030380240F3
:10100000000802400000024000040240000C0240C0
:101010000C4810B50A4901604FF4E13141600021EC
:1010200081600C22C160C0E904128161C161FFF7D7
:10103000B3FE002803D0BDE81040FFF758BA10BD3A
:10104000001001404C0000200C4810B50A49016016
:101050004FF4E1314160002181600C22C160C0E9A0
:1010600004128161C161FFF797FE002803D0BDE83B
:101070001040FFF73CBA10BD004400409000002033
:101080000C4810B50A4901604FF4E131416000217C
:1010900081600C22C160C0E904128161C161FFF767
:1010A0007BFE002803D0BDE81040FFF720BA10BD3A
:1010B00000140140D4000020FEE7FEE710B5FFF762
:1010C00027FB00F091F9012803D0BDE8104000F0A3
:1010D00075B910BD30B593B030216846FFF7A1F95E
:1010E00014210CA8FFF79DF91D480024016841F068
:1010F00080510160006800F080501190194801682B
:1011000021F4404141F4004101600068022500F4EF
:101110004040119001200390102004900095069506
:101120000820CDE907405420CDE9090504200B90A3
:101130006846FFF767FC08B172B6FEE70F20CDE9FD
:101140000C054FF48050CDE90E4002210CA81094FC
:10115000FFF76EFB002801D072B6FEE713B030BD7A
:1011600040380240007000400248016841F47001BC
:101170000160704788ED00E070B5044600680169C1
:10118000E26821F44051114301612169A068E269DC
:1011900008436169114308432168CA6849F20C6336
:1011A0009A430243CA6020684169A26921F44071F0
:1011B0001143416131492068884202D03049884258
:1011C00002D1FFF7DFFB01E0FFF7CCFBE269002370
:1011D000192164253226B2F5004F626828D0A0FBA1
:1011E0000101930F9200FFF7A5F80146B0FBF5F05F
:1011F0006FF01802504301EB800006EB0010B0FBCB
:10120000F5F000F0F002B1FBF5F002EB0012B1FBDB
:10121000F5F06FF01803584301EB800006EB001067
:10122000B0FBF5F000F00F0021681044886070BD3D
:10123000A0FB010192185B41FFF77CF80146B0FB6F
:10124000F5F00201B1FBF5F06FF01803584301EB24
:10125000800006EBC000B0FBF5F000F0F80002EBF8
:101260004002B1FBF5F0584301EB800006EBC000F3
:10127000B0FBF5F000F00700D6E7000000100140D9
:1012800000140140FEE70907090E002804DB00F105
:10129000E02080F80014704700F00F0000F1E0201B
:1012A00080F8141D70470000FFF73AFAFFF712FFAD
:1012B000FFF71CFEFFF7ACFEFFF7C6FEFFF7E0FEF0
:1012C00001220C4E540321463046FFF715FA4FF425
:1012D000FA752846FFF70EF9002221463046FFF73F
:1012E0000BFA2846FFF706F9012221463046FFF7A0
:1012F00003FAEEE7000802400648416B096829B18D
:10130000416BC968C9684968816270474FF0FF3115
:10131000FAE7000010000020D0E9013201699A606C
:10132000D0E901235A604A68824201D182684A604A
:10133000002202610868401E086008687047426821
:101340004A6093688B609368596091600861016896
:10135000491C016070470000164810B5016B11B1BF
:101360000121C16110BD0021C1610169124A01E082
:10137000B9B1491E01EB810352F82330002BF7D09D
:1013800001EB810302EB830202F1080453685B68FE
:101390005360A34201D15B685360DA680260016167
:1013A00010BD502080F31188BFF34F8FBFF36F8FB4
:1013B000FEE70000100000201801002010B55020AA
:1013C00080F31188BFF34F8FBFF36F8F00F01AF8CF
:1013D00018B104494FF080500860002080F3118854
:1013E00010BD000004ED00E00548416919B1006B33
:1013F00018B100207047012070470220704700009C
:10140000100000202DE9F0412E4C0027206B28B160
:10141000A069401CA0613846BDE8F081E668761CF2
:10142000E66013D1606B006838B1502080F31188FA
:10143000BFF34F8FBFF36F8FFEE7606BA16B6163EC
:10144000A063206A401C2062FFF756FFA06ADFF805
:101450007880864209D3606B0068A0B1606BC06879
:10146000C5686868864211D2A0622068C06A00EB35
:10147000800158F82100012800D90127E0690028DF
:10148000C9D00127C7E74FF0FF30EDE7281DFFF770
:1014900043FFA86A18B105F11800FFF73DFFE86A9D
:1014A0002169884200D9206100EB800108EB8100AE
:1014B000291DFFF744FFE86A2168C96A8842CAD338
:1014C0000127C8E710000020180100204FF04070ED
:1014D000E1EE100A70470000000000000000010269
:1014E00003040607080900000000010203040000CD
:1014F00010150008000000204C000000D00100087A
:101500005C1500084C000020F40B0000EC01000802
:101510000100000010000000000000000024F400A2
:1015200000000000000000000000000000000000BB
:1015300000000000000000000000000000000000AB
:10154000000000000000000000000000000000009B
:0C1550000000000000000000000000008F
:040000050800019559
:00000001FF
